:100000000C94B4030C94DC030C94DC030C94DC031C
:100010000C94DC030C94DC030C94DC030C94DC03E4
:100020000C94DC030C94DC030C94DC030C94DC03D4
:100030000C94DC030C94DC030C94DC030C94DC03C4
:100040000C943E1A0C94DC030C94DC030C94DC033B
:100050000C94DC030C94DC030C94DC030C94DC03A4
:100060000C9411190C94DC037E0981098409870919
:100070008A09A0099A099D09204F464600204F4E43
:100080002000457869742020202020202020202076
:100090002020005465737420416C61726D20202013
:1000A0002020200052657365742053657474696E56
:1000B000677320200053637265656E205361766517
:1000C00072202020200053686F772053746172746F
:1000D00073637265656E0042617474657279204164
:1000E0006C61726D202020004C69506F20337320AA
:1000F0004D65746572202020004C69506F2032736A
:10010000204D6574657220202000466C6970205374
:10011000637265656E202020202000352E36352044
:1001200020202020352E382020202020352E393543
:100130000020204368616E6E656C202020205253A1
:10014000534900204D487A005343414E002000207F
:1001500020002000200020204368616E6E656C2026
:100160002020205253534900204D487A00554E46D6
:10017000494E49534845440076312E342062792057
:1001800044766F676F6E656E004359434C4F502B3A
:1001900000E916D516C116AD169916851671165DAD
:1001A00016651678168B169E16B116C416D716EA63
:1001B000164916351621160D16FD16111725173975
:1001C000176C1680169416A816BC16D016E416F8EE
:1001D000161A163F1664168916AE16D316F8161D93
:1001E00017131220112110072208180609190523D8
:1001F0000A1A040B1B03240C1C020D1D25010E1EE4
:10020000000F1F26141527161700000000003E5B84
:100210004F5B3E3E6B4F6B3E1C3E7C3E1C183C7E53
:100220003C181C577D571C1C5E7F5E1C00183C1838
:1002300000FFE7C3E7FF0018241800FFE7DBE7FF34
:1002400030483A060E2629792926407F05050740C1
:100250007F05253F5A3CE73C5A7F3E1C1C08081C82
:100260001C3E7F14227F22145F5F005F5F06097FC0
:10027000017F006689956A606060606094A2FFA259
:100280009408047E040810207E201008082A1C0808
:10029000081C2A08081E101010100C1E0C1E0C3012
:1002A000383E3830060E3E0E06000000000000000A
:1002B0005F00000007000700147F147F14242A7FCA
:1002C0002A12231308646236495620500008070397
:1002D00000001C2241000041221C002A1C7F1C2A15
:1002E00008083E0808008070300008080808080068
:1002F0000060600020100804023E5149453E004263
:100300007F400072494949462141494D3318141232
:100310007F1027454545393C4A494931412111095A
:10032000073649494936464949291E00001400004C
:100330000040340000000814224114141414140066
:100340004122140802015909063E415D594E7C12B2
:1003500011127C7F494949363E414141227F41414A
:10036000413E7F494949417F090909013E414151C7
:10037000737F0808087F00417F41002040413F0112
:100380007F081422417F404040407F021C027F7F53
:100390000408107F3E4141413E7F090909063E4164
:1003A00051215E7F09192946264949493203017FB7
:1003B00001033F4040403F1F2040201F3F40384046
:1003C0003F631408146303047804036159494D43DF
:1003D000007F4141410204081020004141417F0457
:1003E000020102044040404040000307080020543E
:1003F0005478407F2844443838444444283844449E
:10040000287F385454541800087E090218A4A49C6C
:10041000787F0804047800447D40002040403D007F
:100420007F1028440000417F40007C047804787CE1
:10043000080404783844444438FC18242418182448
:100440002418FC7C08040408485454542404043F31
:1004500044243C4040207C1C2040201C3C40304038
:100460003C44281028444C9090907C4464544C4464
:100470000008364100000077000000413608000205
:10048000010204023C2623263C1EA1A161123A402F
:1004900040207A38545455592155557941225454A5
:1004A0007842215554784020545579400C1E5272A0
:1004B000123955555559395454545939555454587D
:1004C0000000457C410002457D420001457C407DA5
:1004D0001211127DF0282528F07C54554500205437
:1004E000547C547C0A097F4932494949323A444490
:1004F000443A324A4848303A4141217A3A4240200F
:1005000078009DA0A07D3D4242423D3D4040403D9F
:100510003C24FF2424487E4943662B2FFC2F2BFFCD
:100520000929F620C0887E0903205454794100002F
:10053000447D413048484A32384040227A007A0AA5
:100540000A727D0D19317D2629292F28262929296E
:100550002630484D402038080808080808080838A0
:100560002F10C8ACBA2F102834FA00007B00000806
:10057000142A142222142A14085500550055AA558D
:10058000AA55AAFF55FF55FF000000FF00101010EC
:10059000FF00141414FF001010FF00FF1010F010E3
:1005A000F0141414FC001414F700FF0000FF00FF07
:1005B0001414F404FC141417101F10101F101F142F
:1005C00014141F00101010F0000000001F10101075
:1005D000101F10101010F010000000FF101010106D
:1005E0001010101010FF10000000FF140000FF009A
:1005F000FF00001F10170000FC04F414141710175C
:100600001414F404F40000FF00F714141414141468
:1006100014F700F7141414171410101F101F1414DB
:1006200014F4141010F010F000001F101F00000050
:100630001F14000000FC140000F010F01010FF1058
:10064000FF141414FF141010101F00000000F0100D
:10065000FFFFFFFFFFF0F0F0F0F0FFFFFF000000F2
:100660000000FFFF0F0F0F0F0F3844443844FC4ABF
:100670004A4A347E02020606027E027E0263554921
:1006800041633844443C04407E201E2006027E0222
:100690000299A5E7A5991C2A492A1C4C7201724CA3
:1006A000304A4D4D303048784830BC625A463D3E65
:1006B000494949007E0101017E2A2A2A2A2A444406
:1006C0005F444440514A444040444A51400000FF86
:1006D0000103E080FF000008086B6B083612362427
:1006E00036060F090F060000181800000010100051
:1006F0003040FF0101001F01011E00191D171200EB
:100700003C3C3C3C000000000000000008000201EE
:1007100000000304070000000000000000010204C4
:100720000810204080010204081020010204081073
:10073000200404040404040404020202020202036A
:100740000303030303000000002300260029000028
:10075000000000250028002B0000000000240027D6
:10076000002A0000030A6F1811241FBECFEFD8E043
:10077000DEBFCDBF15E0A0E0B1E0EAEEFFE302C0CE
:1007800005900D92A63AB107D9F726E0A6EAB5E0A2
:1007900001C01D92A33CB207E1F717E0C8E6D7E01D
:1007A00004C02297FE010E944E1FC436D107C9F72C
:1007B0000E94621D0C94F31F0C940000E82FF0E0DF
:1007C000EF51FE4FE491F0E0EE0FFF1FEF56FE4FAA
:1007D00085919491089581E08093A7051092A805D2
:1007E0008093A9058093AA058093AB051092AC0570
:1007F00008950F931F93CF93DF936091C90580E015
:1008000090E00E94DD1F07EA15E0C0E0D0E0F801AB
:1008100061918F012196CE010E94DD1FC630D10566
:10082000B1F76EEE87E090E0DF91CF911F910F91CD
:100830000C94DD1F0F931F93CF93DF9387E090E01D
:100840000E94D51F8E3EA9F480E090E00E94D51F43
:100850008093C90507EA15E0C1E0D0E0CE010E940F
:10086000D51FF80181938F012196C730D105B1F7CB
:1008700002C080E001C081E0DF91CF911F910F9114
:1008800008950F931F93CF93DF93182F0E94491C55
:10089000019749F1C0E0D0E0812F0E94491C892BCB
:1008A00041F4219665E070E080E090E00E94B71A84
:1008B000F3CF9E01205531092C3D310528F0CC3273
:1008C000D14020F401E003C003E001C004E0C0E037
:1008D000D0E0812F0E94491C019739F42196C9323A
:1008E000D10599F409C080E017C0A89728F4812F9A
:1008F0000E94491C892B11F0802F0EC0812F0E946D
:10090000491C892BD9F382E007C065E070E080E0E4
:1009100090E00E94B71ADDCFDF91CF911F910F9128
:100920000895EF92FF920F931F93CF93DF938C0163
:10093000F12CE12CCCE2D1E08F2D0E94DE03801B54
:10094000910B1816190634F48F2D0E94DE03801BBC
:10095000910B07C08F2D0E94DE039801281B390BD5
:10096000C9018C179D0714F0CE0101C0EF2CF39440
:1009700038E2F31611F0EC01DFCF8E2DDF91CF912D
:100980001F910F91FF90EF9008950F931F93CF93B6
:10099000DF93082F10E2C0E0D0E0802F0E94351BCB
:1009A000C80FD91F1150C9F7CE0125E0969587953C
:1009B0002A95E1F7DF91CF911F910F910895DB0107
:1009C000E82FF0E0EF51FE4FE491E83010F481E4BD
:1009D0000DC0E03110F482E409C0E83110F485E480
:1009E00005C0E03210F486E401C082E58C93E77024
:1009F000EF5C1196EC93119712961C921297CD0111
:100A000008951F93CF93DF93EB01E82FF0E0EF51B0
:100A1000FE4F1491183018F46DE175E011C01031DB
:100A200018F466E275E00CC0183118F46FE275E056
:100A300007C0103218F46CE375E002C066E475E09C
:100A4000CE010E94CE1FDE010D900020E9F7119724
:100A5000AC1BBD0BCE018A0F911DDC0117701F5C12
:100A60001C9311961C92CE01DF91CF911F91089596
:100A70008F5D91409C01369527952F7156E0969594
:100A800087955A95E1F79695982F8827979587959A
:100A9000822B089560E082E00E94131C81E090E0C8
:100AA0000E94F11A61E084E00E94131C81E090E052
:100AB0000E94F11A61E082E00E94131C81E090E044
:100AC0000E94F11A60E082E00E94131C81E090E035
:100AD0000C94F11A60E082E00E94131C81E090E027
:100AE0000E94F11A60E084E00E94131C81E090E013
:100AF0000E94F11A61E082E00E94131C81E090E004
:100B00000E94F11A60E082E00E94131C81E090E0F4
:100B10000C94F11A81E090E00E94F11A60E083E009
:100B20000E94131C81E090E00C94F11A81E090E0A7
:100B30000E94F11A61E083E00E94131C81E090E0C2
:100B40000C94F11A1F93CF93DF930E943805EC01A8
:100B50000E94960581E090E00E94F11A0E948A05A9
:100B60000E944A050E946A050E946A050E946A0561
:100B70000E944A0510E1C0FF03C00E944A0502C05E
:100B80000E946A05D695C7951150A9F70E946A057B
:100B90000E946A050E946A050E946A050E949605E5
:100BA00081E090E00E94F11A60E083E00E94131C53
:100BB00060E082E00E94131C60E084E0DF91CF914E
:100BC0001F910C94131CCF92DF92EF92FF920F9320
:100BD0001F93CF93DF93EC012A96C0FF21968E01DD
:100BE000ECE3DE2EE12CF12C053387E1180718F435
:100BF0000B5F1F4F02C00DE016E1C8010E94A20565
:100C000069E170E080E090E00E94B71A84E10E9400
:100C1000C504E816F90610F4E8017C01DA9451F4F1
:100C20008E01045111096E0124E1C20ED11CE12C88
:100C3000F12C0BC08A3F9105B8F2F2CFE8010E5FAC
:100C40001F4F0C151D0591F07C01C8010E94A205E3
:100C500069E170E080E090E00E94B71A84E10E94B0
:100C6000C504E816F90650F3C701E9CFCE010E948A
:100C7000A205CE01DF91CF911F910F91FF90EF90D0
:100C8000DF90CF900895CF93C3E060E270E086E0FC
:100C90000E94521B68EC70E080E090E00E94B71A5E
:100CA00060E070E086E00E94521B68EB7BE080E031
:100CB00090E00E94B71AC15041F7C3E060E270E0D3
:100CC00086E00E94521B64E670E080E090E00E94A3
:100CD000B71A60E070E086E00E94521B68EE73E095
:100CE00080E090E00E94B71AC15041F7C3E060E293
:100CF00070E086E00E94521B62E370E080E090E0CA
:100D00000E94B71A60E070E086E00E94521B68EC17
:100D100070E080E090E00E94B71AC15041F760E0B7
:100D200070E086E0CF910C94521B9F92AF92BF92DD
:100D3000CF92DF92EF92FF920F931F93CF93DF93A7
:100D4000942EC62FD0E0A82EB12C650183E0C80EEA
:100D5000D11CE091CB05F091CC050484F585E02D04
:100D6000EE24E394F12C02E010E024E030E0AE0148
:100D7000B6018BEC95E00995E091CB05F091CC059F
:100D8000AE014E5F5F4F0484F585E02D04E110E075
:100D90002AE030E0B5018BEC95E00995E091CB05B8
:100DA000F091CC05AE014C5F5F4FB5016E5F7F4F98
:100DB0000484F585E02DE12CF12C00E110E026E023
:100DC00030E08BEC95E0099585E58915B0F4E0916C
:100DD000CB05F091CC050484F585E02DEE24E39459
:100DE000F12C02E010E024E030E0AE014B5F5F4FF9
:100DF000B6018BEC95E0099503C081E48915B0F448
:100E0000E091CB05F091CC050484F585E02DEE242E
:100E1000E394F12C02E010E024E030E0AE01485F02
:100E20005F4FB6018BEC95E0099503C08DE2891503
:100E3000B0F4E091CB05F091CC050484F585E02D6C
:100E4000EE24E394F12C02E010E024E030E0AE0167
:100E5000455F5F4FB6018BEC95E0099503C089E1D2
:100E60008915B0F4E091CB05F091CC050484F585AB
:100E7000E02DEE24E394F12C02E010E024E030E0D9
:100E8000AE01425F5F4FB6018BEC95E0099503C060
:100E900085E08915A8F4E091CB05F091CC05AE0171
:100EA0004F5E5F4F0484F585E02DEE24E394F12C32
:100EB00002E010E024E030E0B6018BEC95E009950B
:100EC000DF91CF911F910F91FF90EF90DF90CF9026
:100ED000BF90AF909F900895CF92DF92EF92FF92D4
:100EE0000F931F93CF93DF939091A9058091A8054D
:100EF000911103C0882309F470C0811105C003E873
:100F000012E0C7E2D2E004C00DEA11E0CFE6D1E082
:100F10008FE00E94C5048017910708F049C0C817E8
:100F2000D90710F5BC016C1B7D0B80E090E00E949E
:100F3000061E6B017C01B8016C1B7D0B80E090E00C
:100F40000E94061E9B01AC01C701B6010E94721DE2
:100F500020E030E048EC52E40E94941E0E94DA1D2A
:100F6000462F653010F00AC040E082E390E0909395
:100F7000B0058093AF0588EC90E00AC06F3068F44C
:100F800084E690E09093B0058093AF0588EE93E0FF
:100F90009093AE058093AD0514C0693150F488EC90
:100FA00090E09093B0058093AF0588EB9BE0F0CF85
:100FB00043E61092B0051092AF051092AE05109264
:100FC000AD0560E28AE3DF91CF911F910F91FF9011
:100FD000EF90DF90CF900C949506DF91CF911F9109
:100FE0000F91FF90EF90DF90CF900895BF92CF9236
:100FF000DF92EF92FF920F931F93CF93DF93CDB7C2
:10100000DEB766970FB6F894DEBF0FBECDBFB82E21
:101010006B018BEC95E00E94B91061E070E08BEC05
:1010200095E00E94801740E050E06AE070E08BECB1
:1010300095E00E94741763E08BEC95E00E947A17AC
:101040008B2D0E94DE03BC014AE050E08BEC95E062
:101050000E94351D47E050E06BE470E08BEC95E0BA
:101060000E94741762E08BEC95E00E947A1768E6A4
:1010700071E08BEC95E00E94B01CE091CB05F09103
:10108000CC050680F781E02DEE24E394F12C08E1F5
:1010900010E02FE730E048E150E060E070E08BECDA
:1010A00095E009954BE150E060E070E08BEC95E055
:1010B0000E94741761E08BEC95E00E947A1766E558
:1010C00071E08BEC95E00E94B01C47E250E060E0DC
:1010D00070E08BEC95E00E94741762E08BEC95E079
:1010E0000E947A1764E571E08BEC95E00E94B01CD9
:1010F00062E571E08BEC95E00E94B01C8E010F5F01
:101100001F4FB8018B2D0E94DF04BC018BEC95E0D2
:101110000E94D31C6FE471E08BEC95E00E94B01C40
:101120004AE050E0B6018BEC95E00E94351D49E3A2
:1011300050E060E070E08BEC95E00E94741761E095
:101140008BEC95E00E947A17B8018B2D0E94010567
:10115000F80101900020E9F7C8018E1B9F0B46960D
:1011600096958795D82EE12CF12CDE1451F06DE484
:1011700071E08BEC95E00E94B01C8FEFE81AF80A42
:10118000F4CFB8018BEC95E00E94D31C0E946C0751
:101190008BEC95E00E944E1266960FB6F894DEBF77
:1011A0000FBECDBFDF91CF911F910F91FF90EF90B8
:1011B000DF90CF90BF900895EF92FF920F931F930F
:1011C0008BEC95E00E94B91061E070E08BEC95E04B
:1011D0000E94801740E050E06AE070E08BEC95E000
:1011E0000E94741763E08BEC95E00E947A1768E424
:1011F00071E08BEC95E00E94B01C47E050E06BE49E
:1012000070E08BEC95E00E94741762E08BEC95E047
:101210000E947A1763E471E08BEC95E00E94B01CA9
:10122000E091CB05F091CC050680F781E02DEE240E
:10123000E394F12C08E110E02FE730E048E150E0C2
:1012400060E070E08BEC95E009954BE150E060E0E8
:1012500070E08BEC95E00E94741761E08BEC95E0F8
:101260000E947A1761E371E08BEC95E00E94B01C5C
:101270000E946C078BEC95E01F910F91FF90EF900F
:101280000C944E121F93CF93DF93182F8BEC95E0A5
:101290000E94B91040E050E060E070E08BEC95E017
:1012A0000E94741761E08BEC95E00E947A1711237D
:1012B00019F0CFEFC10F01C0C8E0D6E0C93008F087
:1012C000C0E0C11305C041E050E060E070E004C040
:1012D00040E050E061E070E08BEC95E00E94861702
:1012E0004C2F50E0FA013197E830F10520F4EC5C26
:1012F000FF4F0C944C1F6AE071E00EC069EF70E084
:101300000BC068EE70E008C067ED70E005C066ECE9
:1013100070E002C065EB70E08BEC95E00E94B01CC1
:10132000EC2FF0E0E955FA4F80818823B1F06DE7AA
:1013300070E015C064EA70E005C063E970E002C0C7
:1013400062E870E08BEC95E00E94B01C60E575E00F
:101350008BEC95E00E94D31C06C068E770E08BEC34
:1013600095E00E94B01C8BEC95E00E94D51CCF5FED
:10137000D15009F0A3CF8BEC95E0DF91CF911F9175
:101380000C944E12CF9380E00E94420985E00E94A7
:101390004104C0E08C2F0E94420985E00E94410474
:1013A000823059F018F4813021F0F4CF853048F0C4
:1013B000F1CFCF5FC93069F3EDCFCC23C1F0C1507D
:1013C000E9CFC630B1F0C73019F40E94EB03E2CF89
:1013D000C83019F40E944306DDCFEC2FF0E0E95548
:1013E000FA4F81E09081911180E08083D3CFC8E0F3
:1013F000D1CFCF9108958BEC95E00E94B9108BEC82
:1014000095E00C944E1264E08BEC95E00C94A010E7
:101410000F931F93CF93DF931FE1115031F185E0BC
:101420000E94491C892B69F1CBEFD0E02197C1F0D4
:1014300060E870E080E090E00E943B1D062F60E4D1
:1014400070E080E090E00E943B1D462F50E0602F4E
:1014500070E020E030E08BEC95E00E94E90FE6CFF1
:101460008BEC95E00E944E12D8CF8BEC95E00E9459
:10147000B9108BEC95E0DF91CF911F910F910C94F7
:101480004E12DF91CF911F910F910895EF92FF922D
:101490000F931F93CF938BEC95E00E94B910E091CE
:1014A000CB05F091CC050680F781E02DEE24E39486
:1014B000F12C00E010E02FE730E040E050E060E089
:1014C00070E08BEC95E0099561E070E08BEC95E0C5
:1014D0000E94801744E050E061E070E08BEC95E002
:1014E0000E94741763E08BEC95E00E947A1769E81C
:1014F00071E08BEC95E00E94B01CE091CB05F0917F
:10150000CC050680F781E02D0BE110E02FE730E0FD
:101510004BE150E060E070E08BEC95E0099543E230
:1015200050E06FE070E08BEC95E00E94741761E092
:101530008BEC95E00E947A1768E771E08BEC95E000
:101540000E94B01C42E350E061E270E08BEC95E059
:101550000E9474176DE671E08BEC95E00E94B01C60
:101560008BEC95E00E944E12C8EC85E00E94491C6D
:10157000892B79F06AE070E080E090E00E94B71A71
:10158000C15099F7CF911F910F91FF90EF900C945C
:10159000080ACF911F910F91FF90EF90089561E09D
:1015A0008DE00E94DA1B61E08DE00E94131C60E078
:1015B00085E00E94DA1B62E085E00E94131C61E076
:1015C00086E00E94DA1B61E083E00E94DA1B61E0A2
:1015D00084E00E94DA1B61E082E00E94DA1B0E9434
:1015E0001A04811104C01092C9050E94EB03809176
:1015F000C9050E94DE030E94A20521E04CE362E0DF
:101600008BEC95E00E9434118BEC95E00E94B910B0
:101610008091A705882329F062E08BEC95E00E9479
:101620008F178BEC95E00E944E1285E00E94491CBA
:10163000892B69F40E94C2090E94F9038091A705D1
:10164000882329F062E08BEC95E00E948F1780914F
:10165000AB0581110E94460A0E94881A605F784D8E
:101660008F4F9F4F6093C2057093C3058093C4054D
:101670009093C50508950F931F93CF93DF93C62FC3
:10168000DEE0D80F8091A60526E330E0281B310963
:1016900060910A0170E000E010E040E050E08BEC67
:1016A00095E00E94AE0E6D2F70E001E010E026E3A1
:1016B00030E040E050E08BEC95E00E94AE0ED0931D
:1016C0000A01C63320F085E38093A60502C0C093CB
:1016D000A6058BEC95E0DF91CF911F910F910C94B3
:1016E0004E12EF92FF920F931F938BEC95E00E94A6
:1016F000B910E091CB05F091CC050680F781E02D83
:10170000EE24E394F12C07E310E02FE730E047E309
:1017100050E060E070E08BEC95E0099561E070E0EE
:101720008BEC95E00E94801761E08BEC95E00E94C5
:101730007A1749E350E060E070E08BEC95E00E949E
:1017400074176BE171E08BEC95E00E94B01C60E0D7
:1017500080E01F910F91FF90EF900C943B0B9F92B4
:10176000AF92BF92CF92DF92EF92FF920F931F93AF
:10177000CF93DF935C010E94710BCA2DDB2D0AE031
:1017800010E079E3E72E77E1F72EE3E0CE2ED12CBF
:10179000F4E69F2E85E00E944104811127C0239624
:1017A000CA3387E1D80710F0CDE0D6E1CE010E9420
:1017B000A20569E170E080E090E00E94B71A84E140
:1017C0000E94C5048C589109B8010E94F71E262F6B
:1017D000C7018C1B9D0BB6010E94F71E862F622F3E
:1017E000992D981B892F0E943B0BD4CF8E01045159
:1017F00011096496E12CF12CC8010E94A20569E14F
:1018000070E080E090E00E94B71A84E10E94C50475
:10181000E816F90610F0C70101C058010E5F1F4F0E
:101820000C171D0711F07C01E7CFC5010E94A2052E
:10183000C501DF91CF911F910F91FF90EF90DF9045
:10184000CF90BF90AF909F900895CF92DF92EF928C
:10185000FF9285E00E9441048093CA058230B9F16D
:1018600018F4813061F145C0833051F0843009F0C3
:1018700040C08091C9050E94DE030E94AF0B08C0E2
:101880000E94DC088091C9050E94DE030E94E305E6
:101890000E9491048093C90560E070E00E94F60701
:1018A0000E94881A675E7F4F8F4F9F4F6093BE05DF
:1018B0007093BF058093C0059093C1051AC08091B5
:1018C000C905873210F48F5F08C080E006C08091A0
:1018D000C9058150873208F087E28093C9050E94CC
:1018E000DE030E94A20560E070E08091C9050E94BD
:1018F000F6078091CA05882371F00E94881A605FFC
:10190000784D8F4F9F4F6093C2057093C3058093AE
:10191000C4059093C5050E94881AC090BE05D0905A
:10192000BF05E090C005F090C105C616D706E806D1
:10193000F906B8F48091AC05882309F4A2C0C090E0
:10194000C205D090C305E090C405F090C5050E9483
:10195000881AC616D706E806F90608F092C00E9453
:10196000FB099091C9058091C805981781F00E94E4
:10197000881AC090BA05D090BB05E090BC05F090E5
:10198000BD05C616D706E806F90608F495C00E94FC
:10199000881AC090B605D090B705E090B805F090D1
:1019A000B905C616D706E806F906A8F481E09091B5
:1019B0000B01911180E080930B010E94881A6C50FA
:1019C0007E4F8F4F9F4F6093B6057093B7058093FE
:1019D000B8059093B90560910B018DE00E94131C2E
:1019E0008091AA05882309F443C08091AF059091A6
:1019F000B005892BE9F10E94881AC090B205D090F9
:101A0000B305E090B405F090B505C616D706E80614
:101A1000F90608F066C081E09091B105911180E06F
:101A20008093B105882361F060E270E086E00E9457
:101A3000521B0E94881A2091AF053091B0050BC04F
:101A400060E070E086E00E94521B0E94881A20919C
:101A5000AD053091AE05620F731F811D911D60931E
:101A6000B2057093B3058093B4059093B50539C062
:101A700060E070E086E0FF90EF90DF90CF900C94F4
:101A8000521B84E10E94C5049093C7058093C6054C
:101A9000BC018091C9050E94F6070E94881A68510E
:101AA0007C4F8F4F9F4F6093BE057093BF0580930F
:101AB000C0059093C10555CF0E94F9038091C905D7
:101AC0008093C8050E94881A605F784D8F4F9F4FA2
:101AD0006093BA057093BB058093BC059093BD05D8
:101AE00056CFFF90EF90DF90CF9008950F931F9304
:101AF000CF93DF93EC018D89823061F08330D9F090
:101B0000813009F0C8C0EC81FD81E41BF50B3197F1
:101B1000DB0118C08C819D81DC01A61BB70BBD01C8
:101B20008E819F81FC01E41BF50BAF0141505109EF
:101B3000621B730BB0C0AE81BF81A61BB70BA21B8B
:101B4000B30BFA01F7FD05C18C819D81E817F907F8
:101B50000CF0FFC0B7FF04C02A0F3B1FA0E0B0E0AD
:101B60008E819F81AD01420F531F841795071CF48E
:101B70009C012A1B3B0B121613060CF0EAC0422FE5
:101B80008A2F86958695869590E8899FE00DF11DB0
:101B90001124E45EFE4FA77069F158E05A1B852FAF
:101BA00090E0EC01CC5EDE4F6881251760F4DC012B
:101BB000A21BB1098FEF90E00A2E02C09595879580
:101BC0000A94E2F768230130110539F048F0023039
:101BD000110551F48081862706C08081862B03C0C1
:101BE0006095808186238083451708F4B2C0451B29
:101BF000E058FF4F4830A0F102301105A9F4DF0191
:101C0000842F9C9190959C93A058BF4F885088300A
:101C1000C0F788EF840F869586958695B0E88B9FF0
:101C2000E00DF11D112419C081E00130110509F00A
:101C300080E0982F9195EF01842F9883C058DF4F53
:101C400088508830D0F788EF840F869586958695E2
:101C500090E8899FE00DF11D1124E058FF4F477077
:101C6000442309F476C0A42FB0E0A45FBE4F9C913A
:101C70000130110541F050F00230110509F069C042
:101C80008081892706C08081892B03C0909580813F
:101C9000892380835EC057FD5CC08E819F81481779
:101CA00059070CF056C077FF04C0260F371F60E0BD
:101CB00070E08C819D81FB01E20FF31F8E179F075F
:101CC0001CF49C01261B370B121613060CF041C0A6
:101CD000CA0157FD0796E3E095958795EA95E1F7E8
:101CE0009695982F882797958795845E9E4F860FA7
:101CF000971F4770552761E070E001C0660F4A9555
:101D0000EAF7462F0130110541F088F00230110545
:101D100001F5FC01280F391F15C0FC01280F391FE0
:101D2000E217F307B1F08081842B8193F9CF60959E
:101D3000FC01280F391FE217F30759F08081862331
:101D40008193F9CFE217F30721F0808184278193F3
:101D5000F9CFDF91CF911F910F9108950F931F93AA
:101D6000CF93DF93FC018589823069F08330E1F005
:101D7000813009F082C0C481D581C41BD50BC21B40
:101D8000D30BDB0117C084819581DC01A61BB70B47
:101D9000BD016150710986819781DC01A41BB50BDF
:101DA000AD01421B530B69C0A681B781A61BB70BBF
:101DB0001197EA01B7FD08C186819781A817B90775
:101DC0000CF002C1D7FF04C02C0F3D1FC0E0D0E0D3
:101DD00084819581AE01420F531F841795071CF42F
:101DE0009C012C1B3D0B121613060CF0EDC0CD010F
:101DF000B7FD079643E0959587954A95E1F7969547
:101E0000982F882797958795845E9E4F8C0F9D1FEE
:101E1000A770BB2741E050E00A2E01C0440F0A948E
:101E2000EAF7642F0130110549F098F002301105EE
:101E300009F0CAC0FC01280F391F17C0FC01280F88
:101E4000391FE217F30709F4BFC08081862B819305
:101E5000F8CF4095FC01280F391FE217F30709F46A
:101E6000B3C0808184238193F8CFE217F30709F48C
:101E7000ABC0808186278193F8CF77FDA5C0848190
:101E80009581681779070CF09FC057FF04C0240F95
:101E9000351F40E050E086819781FA01E20FF31F81
:101EA0008E179F071CF49C01241B350B121613067A
:101EB0000CF08AC0522F842F869586958695FB015B
:101EC000B0E88B9FE00DF11D1124E45EFE4F4770DA
:101ED00069F168E0641B862F90E0EC01CC5EDE4F78
:101EE0004881261760F4DC01A21BB1098FEF90E056
:101EF0000A2E02C0959587950A94E2F7482301308F
:101F0000110539F048F00230110551F48081842721
:101F100006C08081842B03C0409580818423808308
:101F2000561708F451C0561BE058FF4F5830A0F127
:101F300002301105A9F4DF01852F9C9190959C93A7
:101F4000A058BF4F88508830C0F788EF850F86951E
:101F500086958695B0E88B9FE00DF11D112419C080
:101F600081E00130110509F080E0982F9195EF0193
:101F7000852F9883C058DF4F88508830D0F788EF7E
:101F8000850F86958695869590E8899FE00DF11DD1
:101F90001124E058FF4F57705523B1F0A52FB0E042
:101FA000A45FBE4F9C910130110539F048F002301A
:101FB000110551F48081892706C08081892B03C0D7
:101FC0009095808189238083DF91CF911F910F911C
:101FD0000895CF92DF92EF92FF920F931F93CF93CA
:101FE000DF937C018B01EA01690177FDA0C00E94AB
:101FF000A417081719070CF09AC0D7FD98C0C7019D
:102000000E94A817C817D9070CF091C0C7010E94F9
:102010008C17823009F07FC0F701848195819C0183
:10202000201B310B89010150110986819781FC0128
:10203000EC1BFD0BEF0121970BC0813049F4F70138
:10204000848195818C1B9D0BE8018C010150110945
:10205000F1E0CF16D10431F010F132E0C316D10413
:10206000E1F165C0FE01D7FD379683E0F595E79570
:102070008A95E1F7F695FE2FEE27F795E795E00FA5
:10208000F11FE45EFE4FC770DD2781E090E00C2E6B
:1020900001C0880F0A94EAF79081982B3AC0FE019C
:1020A000D7FD3796A3E0F595E795AA95E1F7F69564
:1020B000FE2FEE27F795E795E00FF11FE45EFE4F48
:1020C000C770DD2781E090E00C2E01C0880F0A94D4
:1020D000EAF78095908198231CC0FE01D7FD3796C2
:1020E00063E0F595E7956A95E1F7F695FE2FEE2703
:1020F000F795E795E00FF11FE45EFE4FC770DD270F
:1021000081E090E00C2E01C0880F0A94EAF79081DC
:10211000982790830CC0833009F08FCFF701868118
:102120009781801B910B8E01EC01219791CFDF915C
:10213000CF911F910F91FF90EF90DF90CF90089576
:102140001F93CF93DF93EC01162F40E450E060E83B
:1021500070E00E94DB1489E595E0998388838FEF16
:102160008C8F88A38E8F8D8F1F8FDF91CF911F91C2
:10217000089580E094E0ECE1F1E0DF019C011D9224
:1021800021503040E1F70895FC0181A1882339F006
:102190006EBD00000DB407FEFDCF8EB5089588E03A
:1021A00090E030E8A4A1B5A14C9123A5209524236B
:1021B0002C93A2A1B3A122A5432F462321F04C9139
:1021C000422B4C9304C04C91209524232C93A4A122
:1021D000B5A12C9143A5242B2C933695019711F78B
:1021E00008951F93CF93DF93EC01162F8C8D8F3FB3
:1021F00009F1EEA1FFA180819CA5892B8083E8A530
:10220000F9A590818DA5809589238083EEA1FFA1FA
:1022100090818CA5809589238083CE010E94C41073
:10222000EEA1FFA180819CA5892B8083DF91CF91B6
:102230001F9108958A8D682F772767FD70958AEF23
:1022400095E00E94571860E08AEF95E00E9404181C
:10225000612F8AEF95E00E9404188AEF95E0DF91E4
:10226000CF911F910C946C180F931F93CF93DF9312
:10227000EC01162F022F6B8F4A8F8C8D8F3F09F444
:1022800077C061E08E8D0E94DA1B61E088A10E9418
:10229000DA1B88A1992787FD9095FC01EF5CF84F28
:1022A000E491F0E0EE0FFF1FE15BF84F25913491D0
:1022B0003FA32EA3FC01E35EF84F84918CA78E8D83
:1022C000992787FD9095FC01EF5CF84FE491F0E0D1
:1022D000EE0FFF1FE15BF84F2591349139A728A736
:1022E000FC01E35EF84F84918DA789A1811134C070
:1022F00061E08C8D0E94DA1B61E08D8D0E94DA1BFB
:102300008D8D992787FD9095FC01EF5CF84FE49146
:10231000F0E0EE0FFF1FE15BF84F259134913DA3F4
:102320002CA3FC01E35EF84F84918BA78C8D992739
:1023300087FD9095FC01EF5CF84FE491F0E0EE0F23
:10234000FF1FE15BF84F259134913BA32AA3FC01C9
:10235000E35EF84F84918AA789A1882369F00E94DF
:102360001E138CB58C7F8CBD8DB581608DBD04C076
:102370008AEF95E00E9443180023E1F061E08F8D21
:102380000E94DA1B61E08F8D0E94131C61E070E0F7
:1023900080E090E00E94B71A60E08F8D0E94131CCD
:1023A0006AE070E080E090E00E94B71A61E08F8DF3
:1023B0000E94131C6EEACE010E94F11065EDCE0161
:1023C0000E94F11060E8CE010E94F11068EACE018F
:1023D0000E94F1106FE3CE010E94F11063EDCE0177
:1023E0000E94F11060E0CE010E94F11060E4CE0185
:1023F0000E94F1106DE8CE010E94F110113011F42D
:1024000060E101C064E1CE010E94F11060E2CE0102
:102410000E94F11060E0CE010E94F11061EACE014D
:102420000E94F11068ECCE010E94F1106AEDCE011D
:102430000E94F11062E1CE010E94F11061E8CE012C
:102440000E94F110113011F46FE901C06FECCE0160
:102450000E94F11069EDCE010E94F110113011F4CB
:1024600062E201C061EFCE010E94F1106BEDCE017E
:102470000E94F11060E4CE010E94F11064EACE01E6
:102480000E94F11066EACE010E94F1106FEACE01BF
:10249000DF91CF911F910F910C94F1106F927F9269
:1024A0008F929F92AF92BF92CF92DF92EF92FF9264
:1024B0000F931F93CF93DF93EC0160E00E94F11024
:1024C00060E1CE010E94F11060E4CE010E94F110A3
:1024D0008C8D8F3F09F44FC070EB772EC12CD12C1F
:1024E000672DCE010E94F11062E0CE010E94F11032
:1024F00060E1CE010E94F11000E010E0C601845EB0
:102500009E4F5C01EEA1FFA180819CA5892B808359
:10251000E8A5F9A580819DA5892B8083EEA1FFA167
:1025200090818CA5809589238083E12CF12C450135
:10253000800E911EF401EE0DFF1D6081CE010E9400
:10254000C4109FEFE91AF90A80E1E816F10491F747
:10255000EEA1FFA180819CA5892B8083005F1F4F86
:102560000038110579F690E8C90ED11C739488EBF8
:102570007812B6CF54C06090B8008CE08093B80059
:1025800060EB762EC12CD12C672DCE010E94F1106C
:1025900062E0CE010E94F11060E1CE010E94F110D4
:1025A00000E010E0C601845E9E4F5C016A8D7727D3
:1025B00067FD70958AEF95E00E945718E091FA0543
:1025C000F091FB050190F081E02D60E48AEF95E049
:1025D0000995E12CF12C4501800E911EF401EE0DC0
:1025E000FF1D60818AEF95E00E9404189FEFE91AB1
:1025F000F90A80E1E816F10489F78AEF95E00E9474
:102600006C18005F1F4F0038110581F690E8C90E65
:10261000D11C739488EB7812B7CF6092B800DF9129
:10262000CF911F910F91FF90EF90DF90CF90BF90CF
:10263000AF909F908F907F906F900895CF93CFB77A
:10264000F8948091F905811127C0EBE3F7E08491BC
:10265000E7E2F7E09491E82FF0E0EE0FFF1FE75A72
:10266000F84FA591B4918C91892321F461E08AE01F
:102670000E94131C61E08AE00E94DA1B8CB5806125
:102680008CBD8CB580648CBD61E08DE00E94DA1B4E
:1026900061E08BE00E94DA1B8091F9058F5F8093E7
:1026A000F905CFBFCF9108952F923F924F925F923D
:1026B0006F927F928F929F92AF92BF92CF92DF9252
:1026C000EF92FF920F931F93CF93DF9300D000D030
:1026D000CDB7DEB74C017C836B836A015901C80119
:1026E0008701AC014C195D0957FF03C05195419515
:1026F000510995016B817C81261B370B37FF03C085
:1027000031952195310922242394312C2417350742
:1027100014F0212C312C2114310459F03A2D2B2D99
:102720005C01832F922F3B812C81DC82CB82C32ED4
:10273000D22EAB81BC81AA16BB065CF43C2D2D2D9C
:102740006C01832F922F3B812C81BC82AB82A32E04
:10275000B22E2501EB81FC814E1A5F0A3C016C18F8
:102760007D0877FE03C0719461947108720157FE71
:1027700003C0FFEFEF1AFF0AF594E794C816D906D5
:102780002CF421E030E03A83298324C06FEF7FEFFF
:102790007A8369831FC0D401ED91FC910480F58197
:1027A000E02D980121143104D9F04B815C81B601F0
:1027B000C4010995E618F708F7FE06C0E981FA8119
:1027C000CE0EDF1EE40CF51C2B813C812F5F3F4FAA
:1027D0003C832B836B817C81A616B706E4F604C08C
:1027E000A6016B817C81E4CF0F900F900F900F902A
:1027F000DF91CF911F910F91FF90EF90DF90CF90DD
:10280000BF90AF909F908F907F906F905F904F9010
:102810003F902F9008956F927F928F929F92AF92E8
:10282000BF92CF92DF92EF92FF920F931F93CF93BD
:10283000DF93EC015B016A0139014801E881F9810C
:102840000284F385E02D87010995E881F981A601CD
:10285000480D591D415051090284F385E02D930123
:10286000B501CE010995E881F9810084F185E02D5B
:102870009401A601B501CE010995E881F981B50160
:10288000660D771D615071090084F185E02D94017A
:10289000A601CE010995DF91CF911F910F91FF9075
:1028A000EF90DF90CF90BF90AF909F908F907F90F0
:1028B0006F900895EF92FF920F931F93DC01ED91BB
:1028C000FC91240F351F215031090680F781E02D3E
:1028D000780189019B0109951F910F91FF90EF905D
:1028E0000895EF92FF920F931F93DC01ED91FC91FD
:1028F000260F371F215031090680F781E02D78011E
:102900008A0109951F910F91FF90EF9008956F92A2
:102910007F928F929F92AF92BF92CF92DF92EF926F
:10292000FF920F931F93CF93DF935C014A016901DC
:102930003801EB01C60ED71ECC15DD0574F4D501A8
:10294000ED91FC910084F185E02D87019301A401B4
:10295000BE01C50109952196EFCFDF91CF911F915F
:102960000F91FF90EF90DF90CF90BF90AF909F902E
:102970008F907F906F900895EF92FF920F931F9327
:10298000DC01ED91FC9111971A960D911C911B970A
:1029900018962D913C9119970684F785E02D7B01BF
:1029A00040E050E060E070E009951F910F91FF90CA
:1029B000EF9008950895FC011382128281E795E05B
:1029C000918380837583648357834683718760878F
:1029D00053874287158A158614861786168621E046
:1029E000248B8FEF9FEF938B828B918B808B268B29
:1029F000178A118E108E08952F923F924F925F92F8
:102A00006F927F928F929F92AF92BF92CF92DF92FE
:102A1000EF92FF920F931F93CF93DF93CDB7DEB763
:102A20006A970FB6F894DEBF0FBECDBF1C01588762
:102A30004F831C870B87FA86E986CC82DC01589687
:102A40004D915C9159974115510509F0A6C0189612
:102A50008D919C911997681779070CF056C11A96B9
:102A60008D919C911B97EF81F885E817F9070CF081
:102A70004CC1D12CCB013C81F6E03F9F800D911DD4
:102A80001124181619060CF040C1C60103E0880F86
:102A9000991F0A95E1F74F815885840F951F1816E5
:102AA00019060CF032C157968C91811103C0203B5E
:102AB00008F02F5F7E876D874B01198219E0A12EE8
:102AC00012E0B12EA61AB70A55E0259FA00CB11C42
:102AD00011248981853039F0ED85FE85EA0DFB1DD5
:102AE00094919A8301C01A826F8078842301A8E0B0
:102AF000AD83BA81B0FF12C0D101ED91FC91BC81D0
:102B0000B13031F40480F581E02D2B853C8518C06F
:102B10000684F785E02DEB84FC841DC0E985FA85E9
:102B20002B853C85E217F307E1F0D101ED91FC9193
:102B3000BC81B13059F40480F581E02D29853A85B6
:102B4000A2016D857E85C10109950BC00684F785BC
:102B5000E02DE984FA8486019601A301B401C10144
:102B60000995EA81E695EA83FD81F150FD836C0CBD
:102B70007D1C2FEF421A520AF111BBCF39813F5F02
:102B800039838C0C9D1C4D855E854F5F5F4F5E8742
:102B90004D87363009F09DCFB8C0FA013496349194
:102BA000329785919491231BA7E02A9F800D911D58
:102BB0001124FA0125913491398B288BFC01459120
:102BC00054915A8F498FFC0132965491598731960E
:102BD000A491AF873196E491FC013596249131960A
:102BE0008491BC81B23050F0622E772467FC7094DF
:102BF000E82FFF27E7FDF095FE87ED87FC81CF2EBC
:102C0000D12C6C9C40016D9C900C7C9C900C1124F0
:102C1000860E971EA12C1982DE8ACD8AAB01420F47
:102C2000511D27FD5A955E834D83AF81B885A80F4E
:102C3000B11D87FDBA95B88FAF8B59818F85581715
:102C400008F063C0852F90E02D853E85280F391F41
:102C50002C9DD0012D9DB00D3C9DB00D1124EF8118
:102C6000F885EA0FFB1FFB83EA836D807E802401D9
:102C7000FA2D2D81F21BFA8B4F89588D480F591F61
:102C80005C8B4B8B9A89960D862D2D81821B398505
:102C90008317B0F5977061F4898D9A8D0196E88954
:102CA000F989298D3A8DE20FF31FB4909A8F898F9D
:102CB000B7FE1DC0D101ED91FC91BC81B13059F43A
:102CC0000480F581E02D2B853C854B895C89B3011F
:102CD000C10109950CC00684F785E02DEB84FC84C6
:102CE000860196014A815B81B201C1010995BB0C45
:102CF000ED89FE894E0E5F1EFFEF6F1A7F0AC2CF6D
:102D0000A30E49814F5F498398CF6A960FB6F89416
:102D1000DEBF0FBECDBFDF91CF911F910F91FF900E
:102D2000EF90DF90CF90BF90AF909F908F907F906B
:102D30006F905F904F903F902F900895AF92BF9209
:102D4000CF92EF92FF920F931F93CF93DF93EC01FB
:102D5000262F888D998D009709F042C06A3069F45A
:102D60002C898E859F8538E0239F800D911D11242D
:102D70009F878E871D861C86ABC06D3009F4A8C066
:102D80008E898823C1F03C898C859D8546E0349FDF
:102D9000800D911D112448855985841795075CF095
:102DA0001D861C868E859F85E8E03E9F800D911DC7
:102DB00011249F878E87EA88FB88088919894E85A8
:102DC0005F856C857D85CC88CE010E94FC142C89A2
:102DD0008C859D85F6E02F9F800D911D112441C0AB
:102DE0006A3079F41D861C864C89FC0136968491E4
:102DF0002E853F85489F200D311D11243F872E874A
:102E000067C06D3009F464C0AC014C5F5F4FFA01DC
:102E10003491631708F45CC03196E491E61708F426
:102E200057C0FA014491362F341BFC013296A5900D
:102E3000B490F7E03F9FA00CB11C1124F50132962D
:102E4000A4913196E491AA2311F0E1110DC0F5018E
:102E50003496A4902C898C859D85A29E800D911D11
:102E600011249D878C8734C0F5013596E4913E8905
:102E7000332309F13C89B0E0AE0FB11DE7FDBA95EF
:102E80003A9FA0013B9F500D11246C857D85460F14
:102E9000571F68857985461757076CF01D861C8675
:102EA000FC01369684914E855F85389F400D511DFB
:102EB00011245F874E87EA88FB88088919894E8527
:102EC0005F856C857D85CC88CE010E94FC14BFCFC8
:102ED00081E090E0DF91CF911F910F91FF90EF90F3
:102EE000CF90BF90AF900895FC0175876487578796
:102EF00046870895611101C061E0FC01648B08956B
:102F0000FC01738B628B718B608B0895FC01718B5C
:102F1000608B538B428B0895FC0185890895FC01D9
:102F20006370658B8481958126813781613039F0AA
:102F3000633029F09187808733872287089531870E
:102F40002087938782870895FC0180859185089565
:102F5000FC0182859385089580912A0690E0209156
:102F60002B06821B9109089520912B0680912A0639
:102F7000281750F4E22FF0E0E45DF94F808190E0F3
:102F80002F5F20932B0608958FEF9FEF0895E09118
:102F90002B0680912A06E81730F4F0E0E45DF94F43
:102FA000808190E008958FEF9FEF08950895CF926C
:102FB000DF92EF92FF920F931F93CF93DF937C01E9
:102FC000CB018A0120910606222389F0EB016B01D7
:102FD000C40ED51ECC15DD0569F06991D701ED91C0
:102FE000FC910190F081E02DC7010995F3CF642F8A
:102FF0000E94E818C801DF91CF911F910F91FF90B7
:10300000EF90DF90CF900895CF93DF931F92CDB7CD
:10301000DEB76983209106062223D1F020910706AE
:10302000203240F021E030E0FC013383228380E055
:1030300090E015C080910806E82FF0E0E75FF94FB7
:10304000998190838F5F809308068093070605C05F
:1030500061E0CE0101960E94E81881E090E00F90B7
:10306000DF91CF910895FC011382128248EE53E064
:1030700060E070E0448355836683778389E895E058
:1030800091838083089510922B0610922A06109245
:103090000806109207060C94731881E080930606C8
:1030A00060932906109208061092070608950C9462
:1030B0004D180F93062F21E04091070669E076E056
:1030C000809129060E949118109208061092070616
:1030D000109206060F91089561E00C9459188AEF3A
:1030E00095E00C9433181092B90681E08093B706EE
:1030F0001092B60661E082E10E94131C61E083E158
:103100000E94131CE9EBF0E080818E7F8083808138
:103110008D7F808380E28093B80085E48093BC003B
:1031200008950F93413208F04AC09091B906911169
:10313000FCCF92E09093B9060093B7069FEF90936F
:103140004C061092910640939006FB0162E976E0EE
:10315000DB019A2F961B941718F491919D93F9CF48
:103160001092B8069091B806880F892B8093B80604
:103170008091B606813061F41092B6068091B8064F
:103180008093BB008091BC0083FDF8CF85EC01C02B
:1031900085EE8093BC00222321F08091B906823015
:1031A000E1F380914C068F3F61F080914C068032B4
:1031B00051F080914C06803341F483E007C081E0F8
:1031C00005C080E003C082E001C084E00F91089553
:1031D000613298F42091B906243089F460936E0628
:1031E000FC0180E796E0DC012A2F281B261718F443
:1031F00021912D93F9CF80E0089581E0089582E038
:10320000089585ED8093BC008091BC0084FDFCCFC7
:103210001092B906089585EC8093BC001092B9060F
:1032200008951F920F920FB60F9211242F933F9380
:103230004F935F936F937F938F939F93AF93BF93BE
:10324000EF93FF938091B900887F803609F49EC088
:1032500078F5883209F45DC090F4803109F456C0E5
:1032600038F4882309F4F5C0883009F44FC0F5C05C
:10327000883109F44EC0803209F45FC0EEC080345A
:1032800009F46AC058F4803309F457C0883309F050
:10329000E4C080934C060E940B19DFC0803509F40E
:1032A0004FC0883509F45DC0883409F0D6C0D3C05A
:1032B000883909F4C4C0A8F4883709F467C038F421
:1032C000883609F463C0803709F460C0C6C0883806
:1032D00009F4B5C0803909F45FC0803809F0BDC079
:1032E0005BC0803B09F483C038F4803A09F466C0BF
:1032F000883A09F47CC0B1C0803C09F4A4C0883C81
:1033000009F4A1C0883B09F487C0A7C08091B80622
:1033100010C09091910680919006981770F5E091F9
:10332000910681E08E0F80939106F0E0EE56F94F02
:1033300080818093BB0085EC83C080934C068BC05A
:10334000E091910681E08E0F809391068091BB0001
:10335000F0E0EE56F94F80839091910680919006AF
:103360006BC0E091910681E08E0F80939106809171
:10337000BB00F0E0EE56F94F80838091B7068111D3
:103380006AC081E08093B60684EA5EC083E08093E1
:10339000B90610924D06CFCF80914D06803208F0CD
:1033A0004EC0E0914D0681E08E0F80934D068091D6
:1033B000BB00F0E0E25BF94F8083BDCF0E940B19A8
:1033C00080914D06803230F4E0914D06F0E0E25BF2
:1033D000F94F108260914D0670E0E091B206F091D5
:1033E000B3068EE496E0099510924D0636C084E04F
:1033F0008093B90610926F0610926E06E091B406A3
:10340000F091B506099580916E06811105C081E0A5
:1034100080936E0610927006E0916F0681E08E0F29
:1034200080936F06F0E0E059F94F80818093BB00F4
:1034300090916F0680916E06981708F47CCF85E80E
:103440008093BC000AC085EC8093BC001092B90642
:1034500004C010924C060E940119FF91EF91BF9198
:10346000AF919F918F917F916F915F914F913F911C
:103470002F910F900FBE0F901F9018951F920F92D3
:103480000FB60F9211242F933F938F939F93AF9377
:10349000BF938091BB069091BC06A091BD06B091F0
:1034A000BE063091BA0626E0230F2D3720F402968F
:1034B000A11DB11D05C029E8230F0396A11DB11D53
:1034C0002093BA068093BB069093BC06A093BD06DA
:1034D000B093BE068091BF069091C006A091C10630
:1034E000B091C2060196A11DB11D8093BF069093B5
:1034F000C006A093C106B093C206BF91AF919F9141
:103500008F913F912F910F900FBE0F901F901895A4
:103510002FB7F8946091BB067091BC068091BD06F0
:103520009091BE062FBF08953FB7F8948091BF06D3
:103530009091C006A091C106B091C20626B5A89B85
:1035400005C02F3F19F00196A11DB11D3FBF662791
:10355000782F892F9A2F620F711D811D911D43E0D5
:10356000660F771F881F991F4A95D1F708958F928C
:103570009F92AF92BF92CF92DF92EF92FF926B0138
:103580007C010E94941A4B015C01C114D104E10436
:10359000F104F1F00E94711D0E94941A68197909D2
:1035A0008A099B09683E73408105910570F321E00B
:1035B000C21AD108E108F10888EE880E83E0981E4F
:1035C000A11CB11CC114D104E104F10429F7DDCF21
:1035D000FF90EF90DF90CF90BF90AF909F908F9033
:1035E00008958330910528F0880F991F049701975B
:1035F000F1F70895789484B5826084BD84B58160C4
:1036000084BD85B5826085BD85B5816085BDEEE6EA
:10361000F0E0808181608083E1E8F0E010828081C9
:1036200082608083808181608083E0E8F0E0808137
:1036300081608083E1EBF0E0808184608083E0EB57
:10364000F0E0808181608083EAE7F0E0808184603F
:10365000808380818260808380818E7F808380816F
:10366000806880831092C10008958E3008F08E50DB
:10367000877020911C0590E4299F90011124822BD2
:1036800080937C0080917A00806480937A0080919E
:103690007A0086FDFCCF809178002091790090E03F
:1036A000922B08951F93CF93DF93182FEB0161E0C6
:1036B0000E94DA1B209711F460E004C0CF3FD105CF
:1036C00039F461E0812FDF91CF911F910C94131C8D
:1036D000E12FF0E0E75FF84FE491E330F9F048F4D0
:1036E000E130B9F0E230A1F584B5806284BDC8BD97
:1036F00034C0E730E9F0E83019F1E43049F5809161
:103700008000806280938000D0938B00C0938A00F9
:1037100024C084B5806884BDC7BD1FC0809180006F
:10372000806880938000D0938900C093880015C082
:103730008091B00080688093B000C093B3000DC04A
:103740008091B00080628093B000C093B40005C047
:10375000C038D1050CF0B5CFAFCFDF91CF911F911D
:103760000895833081F028F4813099F08230A1F0FF
:1037700008958730A9F08830B9F08430D1F4809171
:1037800080008F7D03C0809180008F7780938000C0
:10379000089584B58F7702C084B58F7D84BD089568
:1037A0008091B0008F7703C08091B0008F7D8093AF
:1037B000B0000895CF93DF9390E0FC01E35EF84FF3
:1037C0002491FC01EF5CF84F8491882349F190E04B
:1037D000880F991FFC01E75AF84FA591B491815BBE
:1037E000984FFC01C591D4919FB7611108C0F8941E
:1037F0008C91209582238C93888182230AC0623029
:1038000051F4F8948C91322F309583238C938881D6
:10381000822B888304C0F8948C91822B8C939FBF59
:10382000DF91CF9108950F931F93CF93DF931F9252
:10383000CDB7DEB7282F30E0F901E75FF84F84916C
:10384000F901E35EF84F1491F901EF5CF84F049130
:103850000023C9F0882321F069830E94B11B69818C
:10386000E02FF0E0EE0FFF1FE15BF84FA591B49160
:103870009FB7F8948C91611103C01095812301C00A
:10388000812B8C939FBF0F90DF91CF911F910F9150
:103890000895CF93DF93282F30E0F901E75FF84FC9
:1038A0008491F901E35EF84FD491F901EF5CF84F90
:1038B000C491CC2391F081110E94B11BEC2FF0E058
:1038C000EE0FFF1FEB5BF84FA591B4912C912D23C8
:1038D00081E090E021F480E002C080E090E0DF91A0
:1038E000CF910895CF92DF92EF92FF920F931F93A3
:1038F000CF93DF937C016A01EB0100E010E00C152F
:103900001D0571F06991D701ED91FC910190F08155
:10391000E02DC7010995892B19F00F5F1F4FEFCFDD
:10392000C801DF91CF911F910F91FF90EF90DF9031
:10393000CF9008956115710581F0DB010D90002095
:10394000E9F7AD0141505109461B570BDC01ED91E0
:10395000FC910280F381E02D099480E090E00895CD
:10396000EF92FF920F931F93CF93DF938C017B0114
:10397000C0E0D0E0F701EC0FFD1F6491662359F021
:10398000F801A081B181ED91FC91C8010995892BC5
:1039900011F02196EFCFCE01DF91CF911F910F91C2
:1039A000FF90EF9008950C949A1C65E975E00C94D3
:1039B0009A1C8F929F92AF92BF92DF92EF92FF92EA
:1039C0000F931F93CF93DF93CDB7DEB7A1970FB6B9
:1039D000F894DEBF0FBECDBF7C01F42FD52ECB01F6
:1039E00019A2223008F42AE08E010F5D1F4F822EAB
:1039F000912CA12CB12C6F2F7D2DA50194010E943B
:103A00000B1FF22FD32ECA01015011096A3014F492
:103A1000E0E301C0E7E3E60FD801EC93232B242B6E
:103A2000252B49F7B801C7010E949A1CA1960FB631
:103A3000F894DEBF0FBECDBFDF91CF911F910F91E4
:103A4000FF90EF90DF90BF90AF909F908F90089580
:103A50002115310541F4DC01ED91FC910190F081DB
:103A6000E02D642F09940C94D91C9A01AB0160E0FD
:103A700070E00C94281DCF93DF9300D000D0CDB719
:103A8000DEB79B01AC01611571058105910569F0F7
:103A900069833A834B835C830E94BB1F29813A81EF
:103AA0004B815C810E942D1F03C060E070E0CB0160
:103AB0000F900F900F900F90DF91CF9108950E947B
:103AC000C91F08950E94FA1A0E94611D0E94CF0A20
:103AD000C0E0D0E00E94250C2097E1F30E94000096
:103AE000F9CF08950CD0E6C0DED040F0D5D030F04C
:103AF00021F45F3F19F0C7C0511110C1CAC0EBD00B
:103B000098F39923C9F35523B1F3951B550BBB27A4
:103B1000AA2762177307840738F09F5F5F4F220F51
:103B2000331F441FAA1FA9F333D00E2E3AF0E0E84A
:103B300030D091505040E695001CCAF729D0FE2F96
:103B400027D0660F771F881FBB1F26173707480728
:103B5000AB07B0E809F0BB0B802DBF01FF279358DE
:103B60005F4F2AF09E3F510568F08DC0D7C05F3F80
:103B7000ECF3983EDCF3869577956795B795F795C6
:103B80009F5FC9F7880F911D9695879597F90895BE
:103B9000E1E0660F771F881FBB1F6217730784075A
:103BA000BA0720F0621B730B840BBA0BEE1F88F769
:103BB000E095089598D088F09F5790F0B92F9927F5
:103BC000B751A0F0D1F0660F771F881F991F1AF028
:103BD000BA95C9F712C0B13081F09FD0B1E0089515
:103BE0009CC0672F782F8827B85F39F0B93FCCF396
:103BF000869577956795B395D9F73EF4909580951E
:103C0000709561957F4F8F4F9F4F0895E89409C03D
:103C100097FB3EF490958095709561957F4F8F4FFF
:103C20009F4F9923A9F0F92F96E9BB279395F69515
:103C3000879577956795B795F111F8CFFAF4BB0F93
:103C400011F460FF1BC06F5F7F4F8F4F9F4F16C0F7
:103C5000882311F096E911C0772321F09EE8872F81
:103C6000762F05C0662371F096E8862F70E060E03D
:103C70002AF09A95660F771F881FDAF7880F9695B6
:103C8000879597F9089597F99F6780E870E060E05D
:103C900008959FEF80EC089500240A9416161706E5
:103CA00018060906089500240A941216130614062D
:103CB00005060895092E0394000C11F4882352F090
:103CC000BB0F40F4BF2B11F460FF04C06F5F7F4F48
:103CD0008F4F9F4F089557FD9058440F551F59F02F
:103CE0005F3F71F04795880F97FB991F61F09F3FE9
:103CF00079F087950895121613061406551FF2CF12
:103D00004695F1DF08C0161617061806991FF1CF61
:103D100086957105610508940895E894BB27662788
:103D20007727CB0197F908950BD0C4CFB5DF28F0E2
:103D3000BADF18F0952309F0A6CFABCF1124EECF50
:103D4000CADFA0F3959FD1F3950F50E0551F629FF6
:103D5000F001729FBB27F00DB11D639FAA27F00DE4
:103D6000B11DAA1F649F6627B00DA11D661F829F0B
:103D70002227B00DA11D621F739FB00DA11D621FF0
:103D8000839FA00D611D221F749F3327A00D611D0D
:103D9000231F849F600D211D822F762F6A2F1124EF
:103DA0009F5750408AF0E1F088234AF0EE0FFF1F42
:103DB000BB1F661F771F881F91505040A9F79E3F79
:103DC000510570F060CFAACF5F3FECF3983EDCF373
:103DD000869577956795B795F795E7959F5FC1F7B6
:103DE000FE2B880F911D9695879597F90895AA1B2C
:103DF000BB1B51E107C0AA1FBB1FA617B70710F0D6
:103E0000A61BB70B881F991F5A95A9F78095909507
:103E1000BC01CD010895A1E21A2EAA1BBB1BFD0116
:103E20000DC0AA1FBB1FEE1FFF1FA217B307E40799
:103E3000F50720F0A21BB30BE40BF50B661F771FF1
:103E4000881F991F1A9469F76095709580959095D1
:103E50009B01AC01BD01CF010895052E97FB1EF417
:103E600000940E94441F57FD07D00E940B1F07FCBF
:103E700003D04EF40C94441F5095409530952195F5
